:1000000019C032C031C030C02FC02EC02DC02CC08E
:100010002BC02AC029C028C027C026C025C024C0A4
:1000200023C022C021C020C01FC01EC01DC01CC0D4
:100030001BC01AC011241FBECFEFD2E0DEBFCDBF60
:1000400011E0A0E0B1E0EEECF0E002C005900D920E
:10005000A030B107D9F711E0A0E0B1E001C01D92D6
:10006000A030B107E1F710C0CBCF181619065CF429
:1000700028EE33E02250304012161306DCF30197CD
:1000800018161906ACF30895CFEFD2E0DEBFCDBF4E
:100090008FEB85B980EC84B91BB88FEF8AB981E00A
:1000A00088B917B8C82F88E790E0DFDF8BB1880FD9
:1000B0008BB98BB18823B9F7CBB988E790E0D5DF4E
:0E00C0008BB1880F8BB98BB1882369F7F5CF10
:00000001FF
